BL51 BANKED LINKER/LOCATER V6.22.2.0                                                    10/12/2022  17:14:19  PAGE 1


BL51 BANKED LINKER/LOCATER V6.22.2.0, INVOKED BY:
C:\KEIL_V5\C51\BIN\BL51.EXE .\Release\system_FE81001.obj, .\Release\STARTUP.obj, .\Release\main.obj TO .\Release\Sample_
>> DrvI2C_Slave REGFILE (.\Release\Sample_DrvI2C_Slave.ORC) PRINT (.\Sample_DrvI2C_Slave.m51) RAMSIZE (256) CODE (0X0000
>> -0X1FFF) XDATA (0X8000-0X87FF)


MEMORY MODEL: SMALL


INPUT MODULES INCLUDED:
  .\Release\system_FE81001.obj (SYSTEM_FE81001)
  .\Release\STARTUP.obj (?C_STARTUP)
  .\Release\main.obj (MAIN)
  C:\KEIL_V5\C51\LIB\C51S.LIB (?C_INIT)
  C:\KEIL_V5\C51\LIB\C51S.LIB (?C_IBP)


LINK MAP OF MODULE:  .\Release\Sample_DrvI2C_Slave (SYSTEM_FE81001)


            TYPE    BASE      LENGTH    RELOCATION   SEGMENT NAME
            -----------------------------------------------------

            * * * * * * *   D A T A   M E M O R Y   * * * * * * *
            REG     0000H     0008H     ABSOLUTE     "REG BANK 0"
            DATA    0008H     0002H     UNIT         ?DT?DELAY?MAIN
            DATA    000AH     0001H     UNIT         ?DT?I2CISR?MAIN
            DATA    000BH     0001H     UNIT         ?C?LIB_DATA
            IDATA   000CH     0001H     UNIT         ?STACK

            * * * * * * *  X D A T A   M E M O R Y  * * * * * * *
                    0000H     8000H                  *** GAP ***
            XDATA   8000H     0003H     UNIT         ?XD?MAIN

            * * * * * * *   C O D E   M E M O R Y   * * * * * * *
            CODE    0000H     0003H     ABSOLUTE     
            CODE    0003H     004EH     UNIT         ?PR?IOCONFIG?MAIN
            CODE    0051H     0007H     UNIT         ?C_INITSEG
            CODE    0058H     0001H     UNIT         ?PR?SYSTEMINIT?SYSTEM_FE81001
                    0059H     0002H                  *** GAP ***
            CODE    005BH     0003H     ABSOLUTE     
            CODE    005EH     01B2H     UNIT         ?PR?I2CISR?MAIN
            CODE    0210H     009DH     UNIT         ?C_C51STARTUP
            CODE    02ADH     002EH     UNIT         ?PR?I2C_SLAVE_CONFIG?MAIN
            CODE    02DBH     001CH     UNIT         ?PR?DELAY?MAIN
            CODE    02F7H     0017H     UNIT         ?PR?CLKCONFIG?MAIN
            CODE    030EH     0015H     UNIT         ?PR?MAIN?MAIN



OVERLAY MAP OF MODULE:   .\Release\Sample_DrvI2C_Slave (SYSTEM_FE81001)


SEGMENT
  +--> CALLED SEGMENT
---------------------
?C_C51STARTUP
  +--> ?PR?MAIN?MAIN
BL51 BANKED LINKER/LOCATER V6.22.2.0                                                  10/12/2022  17:14:19  PAGE 2


  +--> ?C_INITSEG

?PR?MAIN?MAIN
  +--> ?PR?CLKCONFIG?MAIN
  +--> ?PR?IOCONFIG?MAIN
  +--> ?PR?I2C_SLAVE_CONFIG?MAIN
  +--> ?PR?DELAY?MAIN

*** NEW ROOT ***************************************************

?PR?I2CISR?MAIN
  +--> ?PR?I2C_SLAVE_CONFIG?MAIN



SYMBOL TABLE OF MODULE:  .\Release\Sample_DrvI2C_Slave (SYSTEM_FE81001)

  VALUE           TYPE          NAME
  ----------------------------------

  -------         MODULE        SYSTEM_FE81001
  C:0000H         SYMBOL        _ICE_DUMMY_
  C:0058H         PUBLIC        SystemInit
  -------         PROC          SYSTEMINIT
  C:0058H         LINE#         38
  C:0058H         LINE#         39
  C:0058H         LINE#         41
  -------         ENDPROC       SYSTEMINIT
  -------         ENDMOD        SYSTEM_FE81001

  -------         MODULE        ?C_STARTUP
  C:0210H         SEGMENT       ?C_C51STARTUP
  I:000CH         SEGMENT       ?STACK
  C:0000H         PUBLIC        ?C_STARTUP
  D:00E0H         SYMBOL        ACC
  D:00F0H         SYMBOL        B
  D:0083H         SYMBOL        DPH
  D:0082H         SYMBOL        DPL
  N:0001H         SYMBOL        IBPSTACK
  N:0100H         SYMBOL        IBPSTACKTOP
  N:0080H         SYMBOL        IDATALEN
  C:0213H         SYMBOL        IDATALOOP
  N:0000H         SYMBOL        PBPSTACK
  N:0100H         SYMBOL        PBPSTACKTOP
  N:0000H         SYMBOL        PDATALEN
  N:0000H         SYMBOL        PDATASTART
  N:0000H         SYMBOL        PPAGE
  N:0000H         SYMBOL        PPAGEENABLE
  D:00A0H         SYMBOL        PPAGE_SFR
  D:0081H         SYMBOL        SP
  C:0210H         SYMBOL        STARTUP1
  N:0000H         SYMBOL        XBPSTACK
  N:0000H         SYMBOL        XBPSTACKTOP
  N:0800H         SYMBOL        XDATALEN
  C:021EH         SYMBOL        XDATALOOP
  N:8000H         SYMBOL        XDATASTART
  C:0000H         LINE#         126
BL51 BANKED LINKER/LOCATER V6.22.2.0                                                  10/12/2022  17:14:19  PAGE 3


  C:0210H         LINE#         133
  C:0212H         LINE#         134
  C:0213H         LINE#         135
  C:0214H         LINE#         136
  C:0216H         LINE#         140
  C:0219H         LINE#         141
  C:021BH         LINE#         145
  C:021DH         LINE#         147
  C:021EH         LINE#         148
  C:021FH         LINE#         149
  C:0220H         LINE#         150
  C:0222H         LINE#         151
  C:0224H         LINE#         170
  C:0227H         LINE#         185
  C:022AH         LINE#         196
  -------         ENDMOD        ?C_STARTUP

  -------         MODULE        MAIN
  C:0000H         SYMBOL        _ICE_DUMMY_
  D:0090H         PUBLIC        P1
  D:00B0H         PUBLIC        P3
  X:8000H         PUBLIC        rx_buf
  D:00A8H         PUBLIC        IE
  C:02DBH         PUBLIC        delay
  D:00B8H         PUBLIC        IP
  C:030EH         PUBLIC        main
  C:005EH         PUBLIC        I2CISR
  D:0098H         PUBLIC        SCON
  C:02F7H         PUBLIC        CLKConfig
  D:0088H         PUBLIC        TCON
  C:02ADH         PUBLIC        I2C_Slave_Config
  D:00C8H         PUBLIC        T2CON
  C:0003H         PUBLIC        IOConfig
  D:00D0H         PUBLIC        PSW
  -------         PROC          DELAY
  -------         DO            
  D:0008H         SYMBOL        i
  -------         ENDDO         
  C:02DBH         LINE#         34
  C:02DBH         LINE#         35
  C:02DBH         LINE#         38
  C:02F6H         LINE#         39
  -------         ENDPROC       DELAY
  -------         PROC          I2CISR
  -------         DO            
  D:000AH         SYMBOL        dir
  -------         ENDDO         
  C:005EH         LINE#         51
  C:007BH         LINE#         56
  C:008FH         LINE#         57
  C:008FH         LINE#         58
  C:0095H         LINE#         60
  C:009FH         LINE#         62
  C:00AAH         LINE#         63
  C:00AAH         LINE#         64
  C:00BBH         LINE#         65
  C:00C6H         LINE#         66
BL51 BANKED LINKER/LOCATER V6.22.2.0                                                  10/12/2022  17:14:19  PAGE 4


  C:00D0H         LINE#         68
  C:00E1H         LINE#         69
  C:00ECH         LINE#         70
  C:00F6H         LINE#         72
  C:0107H         LINE#         73
  C:0112H         LINE#         74
  C:011CH         LINE#         76
  C:0122H         LINE#         77
  C:0125H         LINE#         78
  C:0128H         LINE#         81
  C:0128H         LINE#         82
  C:0132H         LINE#         83
  C:0143H         LINE#         84
  C:014EH         LINE#         85
  C:0154H         LINE#         86
  C:015EH         LINE#         88
  C:016FH         LINE#         89
  C:017AH         LINE#         90
  C:0180H         LINE#         91
  C:018AH         LINE#         93
  C:019BH         LINE#         94
  C:01A6H         LINE#         95
  C:01ACH         LINE#         97
  C:01B2H         LINE#         98
  C:01B5H         LINE#         99
  C:01B5H         LINE#         101
  C:01B5H         LINE#         104
  C:01C6H         LINE#         105
  C:01CCH         LINE#         106
  C:01D2H         LINE#         107
  C:01D2H         LINE#         110
  C:01E3H         LINE#         111
  C:01E9H         LINE#         112
  C:01EFH         LINE#         113
  C:01EFH         LINE#         116
  C:01F5H         LINE#         117
  -------         ENDPROC       I2CISR
  -------         PROC          IOCONFIG
  C:0003H         LINE#         130
  C:0003H         LINE#         131
  C:0003H         LINE#         133
  C:0024H         LINE#         136
  C:003AH         LINE#         137
  C:0050H         LINE#         139
  -------         ENDPROC       IOCONFIG
  -------         PROC          CLKCONFIG
  C:02F7H         LINE#         151
  C:02F7H         LINE#         152
  C:02F7H         LINE#         154
  C:0302H         LINE#         157
  C:030DH         LINE#         159
  -------         ENDPROC       CLKCONFIG
  -------         PROC          I2C_SLAVE_CONFIG
  C:02ADH         LINE#         161
  C:02ADH         LINE#         162
  C:02ADH         LINE#         165
  C:02B3H         LINE#         166
BL51 BANKED LINKER/LOCATER V6.22.2.0                                                  10/12/2022  17:14:19  PAGE 5


  C:02B8H         LINE#         169
  C:02BEH         LINE#         172
  C:02CEH         LINE#         175
  C:02D4H         LINE#         176
  C:02DAH         LINE#         178
  -------         ENDPROC       I2C_SLAVE_CONFIG
  -------         PROC          MAIN
  C:030EH         LINE#         190
  C:030EH         LINE#         191
  C:030EH         LINE#         192
  C:0311H         LINE#         193
  C:0314H         LINE#         194
  C:0317H         LINE#         197
  C:031DH         LINE#         199
  C:0320H         LINE#         201
  -------         ENDPROC       MAIN
  -------         ENDMOD        MAIN

  -------         MODULE        ?C_IBP
  D:000BH         PUBLIC        ?C_IBP
  -------         ENDMOD        ?C_IBP



FUNCTION REGISTER MASKS


FUNCTION . . . . . . REG MASK
-----------------------------

CLKCONFIG. . . . . . @0xe301
DELAY. . . . . . . . @0xf000
I2C_SLAVE_CONFIG . . @0xe300
IOCONFIG . . . . . . @0xe301
MAIN . . . . . . . . @0xf301
SYSTEMINIT . . . . . @0x8000

*** WARNING L16: UNCALLED SEGMENT, IGNORED FOR OVERLAY PROCESS
    SEGMENT: ?PR?SYSTEMINIT?SYSTEM_FE81001

Program Size: data=13.0 xdata=3 code=801
LINK/LOCATE RUN COMPLETE.  1 WARNING(S),  0 ERROR(S)
